:1000000000308A00572C00000A108A100A1182075B
:1000100028340C34013406340A108A100A1182077D
:100020000C343E343E344A344F3447344F343C343D
:100030003C340A344E3455344D34453452344F3404
:10004000203441344C344534413454344F345234E8
:1000500049344F3400340A108A100A1182070C34D4
:1000600050347234653470346134723461346434C1
:100070006F343F340A346F346B3400340A108A1002
:100080000A1182070C34433461347234723465349B
:10009000673461346E3464346F340A344E346934F6
:1000A000763465346C3420342534553400340A10E9
:1000B0008A100A1182070C344E3469347634653460
:1000C0006C342034253455342C34203430342034EE
:1000D00061342034253455340A34543465346D3455
:1000E0002034253455342034703461346C34703409
:1000F000693474346534733400340A108A100A1178
:1001000082070C34533465347534203470346134D0
:100110006C3470346934743465343F34203425349D
:10012000553420340A3420342B34203420342D34F8
:100130004F344B3400340A108A100A1182070C34F1
:100140005034613472346134623465346E347334E3
:1001500021340A3450346134733473346F34753459
:100160002034313420344E346934763465346C3480
:10017000213400340A108A100A1182070C344534E5
:10018000723472346F347534213420344F34203457
:100190006E3475346D34653472346F340A346534BA
:1001A00020344D3465346E346F347234213400346D
:1001B0000A108A100A1182070C34453472347234E2
:1001C0006F347534213420344F3420346E34753418
:1001D0006D34653472346F340A34653420344D34F0
:1001E000613469346F347234213400340A108A1057
:1001F0000A11FD3E03188A0A82000C3456346F340B
:100200006334653420345034653472346434653476
:100210007534213420340A344F3420346334653447
:10022000723474346F3420346534203425345534BA
:1002300000340A148A100A1182070C3443346134E2
:10024000723472346534673461346E3464346F34BC
:100250000A344E346F3476346F3420344A346F3479
:1002600067346F340034423084008313000803196C
:1002700047290130F800F701F70B3C29F80B3B291F
:100280004A30F700F70B42294529800B3929003401
:100290003A0EF039F7000F300605770486000000AB
:1002A0008615522986110034C830B8008610F03007
:1002B000660006150000861500000608060E0F39B8
:1002C000BA0086110000861500000608060E0F39D8
:1002D000B9008611003066003A0EF700F030F705DD
:1002E00077083904F8007808B900B91F8029103060
:1002F000F700F70B79290000B80B7F2980295729CF
:10030000361C86103618861400000611000086116F
:10031000370EB9000F30B9053908BA00482137083F
:100320000F39B900BA004821003400306600861049
:10033000061186110F30C20033210130AB002B08AB
:10034000033C031CAB290330BA0048210530C2002E
:100350003321AB0A9F290230BA004821AB012B0898
:10036000033C031CBC292B080420AC00B6012C085C
:10037000B7005421AB0AAF29842C330BC029C32901
:100380004030B400C429B40101303202B40734084B
:100390008038B500B6013508B70054210034310863
:1003A0000C3A0319DA29063A0319E229023A031929
:1003B000E829ED29B6010130B70054210230C2000E
:1003C0003321F3290130B2000230B300BD21F329FB
:1003D000B6011030B7005421F3290130B6003108BE
:1003E000B7005421F32900342F08A5002E08A400DB
:1003F0002D08A3002C08A20000342030CD00C90134
:10040000CA01CB01CC014408FA004308F9004208B4
:10041000F8004108F7000310771C1C2A4508C9079B
:1004200046080318460FCA0747080318470FCB07AB
:1004300048080318480FCC07CC0CCB0CCA0CC90CCD
:10044000FA0CF90CF80CF70CCD0B0B2A0034F80160
:10045000F901F701FA014008031D312A3F08031989
:100460004B2A1030C1000310BD0DBE0DF70DFA0D63
:1004700040087A02031D3E2A3F087702031C472AE0
:100480003F08F702031CFA034008FA020314F80DB0
:10049000F90DC10B332A00342508C4002408C30019
:1004A0002308C2002208C1004130C800C630C7007E
:1004B0004E30C6006D30C500FD2139307707A200EF
:1004C0007808A300303003183130A3077908A4005E
:1004D000003003180130A4077A08A5000030031883
:1004E0000130A5072408F7002508F800F901FA01F2
:1004F0002508AD002408AC002508BE002408BD0076
:100500007F30C000FF30BF0027227708F8007A084C
:10051000F9000034F701F8012D0803102E18F70731
:10052000F70CF80CAE18F707F70CF80C2E19F707B4
:10053000F70CF80CAE19F707F70CF80C2E1AF707A2
:10054000F70CF80CAE1AF707F70CF80C2E1BF70790
:10055000F70CF80CAE1BF707F70CF80C0034320858
:10056000F80131020318B72A3108F700C32AF7014E
:100570000830B300B10DF70D320877020318F70009
:10058000F80DB30BBA2A003478082F08B100643094
:10059000B200AF227708AF0078083030031DD72AA9
:1005A000B01CDE2AB019DE2A301A2030DA2AB01147
:1005B00030123014F8077808B100CF212F08B100AD
:1005C0000A30B200AF227708AF0078083030031D40
:1005D000EF2AB019F32A301CF32A301A2030F8071A
:1005E0007808B100CF213030AF072F08B100CF21FC
:1005F0000034F701F801F901FA01CE01CF01D00171
:10060000D1014D084C044B044A040319372B203008
:10061000D2000310C60DC70DC80DC90DCE0DCF0DEC
:10062000D00DD10D4D085102031D202B4C08500256
:10063000031D202B4B084F02031D202B4A084E029E
:10064000031C312B4A08CE024B08031C4B0FCF0270
:100650004C08031C4C0FD0024D08031C4D0FD10257
:100660000314F70DF80DF90DFA0DD20B092B4E30CE
:10067000840083130034C1013E0841020318452B56
:10068000FA30C2003321C10A3C2B3D08C20033219D
:10069000C101400841020318532B5330F700F70BF8
:1006A0004F2BC10A492B3F08C2001230C202031C63
:1006B000682B423084008313FC3080050310800CCB
:1006C000800C00080319682B662B0000800B652B3B
:1006D0000034C9010F30C8004230C7004030C600A6
:1006E000CD01CC012C08CB002B08CA00F922031045
:1006F0007A0CC400790CC300780CC200770CC100DE
:100700000A304102AF004208B0000030031C013043
:10071000B0024308B1000030031C0130B1024408AC
:10072000B2000030031C0130B2023208C9003108A7
:10073000C8003008C7002F08C600CD01CC01033027
:10074000CB00E830CA00F9227808B4007708B3007B
:100750003408BE003308BD00C001FA30BF002722B4
:100760007808B8003408BE003308BD00C001FA3074
:10077000BF0027227708B9003208C9003108C80035
:100780003008C7002F08C600CD01CC010330CB00D4
:10079000E830CA00F9220008B500840A0008B60053
:1007A0003608BE003508BD00C001FA30BF00272260
:1007B0007808B7003608BE003508BD00C001FA3021
:1007C000BF0027227708BA00C001BF012E08BE0073
:1007D0002D08BD004008C4003F08C3002E08C20019
:1007E0002D08C100C801C7010330C600E830C500AC
:1007F000FD217A08C1007908C0007808BF00770899
:10080000BE00C9010F30C8004230C7004030C600EA
:10081000CD01CC012C08CB002B08CA00F9227A08A4
:10082000C5007908C4007808C3007708C2004108F1
:10083000C9004008C8003F08C7003E08C6007A0843
:10084000CD007908CC007808CB007708CA00F922DF
:100850007808BC007708BB003C08FA003B08031985
:10086000BC03BB03BD007A08BE00BD08031D3B2CC2
:10087000BE080319562C3908BD003808BE003A08D6
:10088000BF003708C0003B238316061083120614EE
:100890003908BD003808BE003A08BF003708C0005C
:1008A0003B2383160610831206102C2C003484017F
:1008B00083131F30830583168E15073083129F0024
:1008C000A001A10183160108C739083881008312ED
:1008D00090010030F800920000308316920007303B
:1008E00083129F00831605080330F700F70B762C60
:1008F00083121F080C1383169F01003065006600E9
:100900008312850186019529A6010130A7000C30CC
:10091000B100CF210430AB002030B100CF21AB0BB0
:100920008C2C0130AC002C080C20AC0AF700B10074
:10093000CF211A302C02031D932C0C30AB00FA305F
:10094000C2003321AB0B9F2C0130AA002A08103CB7
:10095000031CC02C2A08B2000130B300BD21DB30DB
:10096000B100CF212A08113CAB00B200B301BD2178
:10097000DB30B100CF216430C2003321AA0AA62C9B
:10098000C830C2003321AB012B082B20AB0AF70083
:10099000B100CF210C302B02031DC42C0D30AC0054
:1009A0002030B100CF21AC0BD02C6F30B100CF2163
:1009B0006B30B100CF218316051583120519DB2C8E
:1009C0000108AB00AF01AE01AD012B08AC00F42172
:1009D0004C227908AC007808AB002708AD000A303B
:1009E000AE008A227808AD002C08BE002B08BD009E
:1009F000C0017808BF00272201307707A900AB01AA
:100A00002B083E20AB0AF700B100CF2112302B0299
:100A1000031D002D2708AF001B30B000C4220C308E
:100A2000AB00FA30C2003321AB0B112D0330A8000C
:100A3000A8080319DE2F2708AD000A30AE008A226D
:100A40007808AB00AC012C085720AC0AF700B100C5
:100A5000CF2107302C02031D232D2708AF001B30A8
:100A6000B000C4220930AD002D085720AD0AF700B0
:100A7000B100CF210F302D02031D342D2B08AF0004
:100A80001B30B000C4221130AE002E085720AE0A31
:100A9000F700B100CF2116302E02031D452D280886
:100AA000AF001B30B000C4221830AF002F08572011
:100AB000AF0AF700B100CF2121302F02031D562DC0
:100AC0000C30AB00FA30C2003321AB0B622DAB010E
:100AD0002B087D20AB0AF700B100CF210E302B028E
:100AE000031D682D2608AF001B30B000C422103053
:100AF000AC002C087D20AC0AF700B100CF211730E4
:100B00002C02031D792D0730AD002030B100CF211C
:100B1000AD0B852D4F30B100CF214B30B100CF212F
:100B2000831605158312051DB62D0E30B200013057
:100B3000B300BD212608AF001B30B000C422203016
:100B4000B100CF218316051483120518AC2DA60A17
:100B5000FA30C2003321B52D83168514831285180F
:100B6000B52DA603FA30C2003321902D29082602A4
:100B7000031D782E0230AC000B30AB00AE013230DA
:100B8000AD0069230230AC002A30AB00AE01323038
:100B9000AD0069230230AC004B30AB00AE01323007
:100BA000AD0069230230AC006E30AB00AE013230D4
:100BB000AD0069230330AC001030AB00AE01323021
:100BC000AD0069230230AC00E430AB00AE0132303E
:100BD000AD0069230230AC000B30AB00AE01323007
:100BE000AD0069230230AC002A30AB00AE013230D8
:100BF000AD0069230230AC004B30AB00AE013230A7
:100C0000AD0069230230AC006E30AB00AE01323073
:100C1000AD0069230230AC00E430AB00AE013230ED
:100C2000AD0069230330AC001030AB00AE013230B0
:100C3000AD006923AA012A08033C031C3D2EAB0129
:100C40002B089B20AB0AF700B100CF211A302B02F2
:100C5000031D202E0430AB00AF30C2003321AB0B9C
:100C60002C2E0C30B100CF210430AB00AF30C200CD
:100C70003321AB0B362EAA0A1B2EA70AA60106307B
:100C8000A8000108AB00AF01AE01AD012B08AC001C
:100C9000F4214C227908AC007808AB002708AD009D
:100CA0000A30AE008A227808AD002C08BE002B085E
:100CB000BD00C0017808BF00272201307707A900D6
:100CC000AB012B083E20AB0AF700B100CF21123058
:100CD0002B02031D612E2708AF001B30B000C42279
:100CE0000C30AB00FA30C2003321AB0B722E3B2F1D
:100CF000260829020318DA2E280B7F2EDA2EAB01E4
:100D00002B08BA20AB0AF700B100CF2119302B0213
:100D1000031D802E0130AC002630AB00AE01323016
:100D2000AD0069230230AC009330AB00AE0132302D
:100D3000AD0069230130AC002630AB00AE0132308B
:100D4000AD0069230230AC009330AB00AE0132300D
:100D5000AD0069230130AC002630AB00AE0132306B
:100D6000AD0069230230AC009330AB00AE013230ED
:100D7000AD0069230130AC002630AB00AE0132304B
:100D8000AD0069230230AC009330AB00AE013230CD
:100D9000AD0069230130AC002630AB00AE016430F9
:100DA000AD0069230C30AB00FA30C2003321AB0B2D
:100DB000D42E3B2F2908260203183B2F280BE12EA7
:100DC0003B2FAB012B08D820AB0AF700B100CF2195
:100DD00019302B02031DE22E0130AC002630AB008F
:100DE000AE013230AD0069230230AC009330AB006D
:100DF000AE013230AD0069230130AC002630AB00CB
:100E0000AE013230AD0069230230AC009330AB004C
:100E1000AE013230AD0069230130AC002630AB00AA
:100E2000AE013230AD0069230230AC009330AB002C
:100E3000AE013230AD0069230130AC002630AB008A
:100E4000AE013230AD0069230230AC009330AB000C
:100E5000AE013230AD0069230130AC002630AB006A
:100E6000AE016430AD0069230C30AB00FA30C20033
:100E70003321AB0B362F290826020319DC2F280B50
:100E8000DC2F0130AC003730AB000130AE002C302D
:100E9000AD0069230130AC002630AB000130AE005C
:100EA0009030AD0069230130AC001530AB0001304B
:100EB000AE009030AD0069230130AC000630AB00CD
:100EC0000130AE009030AD0069230130AC00063037
:100ED000AB00AE013230AD0069230130AC001530FB
:100EE000AB00AE013230AD0069230130AC000630FA
:100EF000AB000130AE002C30AD006923AA012A08F6
:100F0000033C031CA62FAB012B08F620AB0AF7000D
:100F1000B100CF2119302B02031D842F2908AF0007
:100F20001B30B000C4220430AB00AF30C20033210C
:100F3000AB0B952F0C30B100CF210430AB00AF309C
:100F4000C2003321AB0B9F2FAA0A7F2F0430A800C9
:100F5000A6010130A7000108AB00AF01AE01AD0151
:100F60002B08AC00F4214C227908AC007808AB00C7
:100F70002708AD000A30AE008A227808AD002C08A0
:100F8000BE002B08BD00C0017808BF002722013039
:100F90007707A900AB012B081921AB0AF700B100B4
:100FA000CF2115302B02031DCB2F0C30AB00FA30B4
:100FB000C2003321AB0BD72FA803182D842C63005C
:02400E00183F59
:00000001FF
